:020000040000FA
:10000000F26A17EF00F0FFFFF9EF0AF0FFFFFFFFC2
:10001000FFFFFFFFFFFFFFFFFBEF0AF0C70ED56EEC
:10002000940ED66EF294F2A413EF00F01200F26A6E
:10003000000E806E896E000E816E8A6E420E826E98
:100040008B6E000E846E170E926E370E936E800EBE
:10005000946E000E966E030EE8CF38FF000EE8CFC8
:1000600039FF000EE8CF3AFF080EE8CFC1FF870E38
:10007000E8CFC0FF000E796E786E776EFD0E616E70
:10008000F19E010EE06E000E9B6E040ED26E080E05
:10009000D36E086A096A0A6A0B6A0C6A0D6A0E6AEC
:1000A0000F6A106A116A0F80AA6B000E2E6F000E85
:1000B000426F000E316F306F3C0E296F000E356FAE
:1000C000A46FA56F3C0E346F336F000E2A6FECECFB
:1000D00020F0D00EB96FBB6F020EBA6FBC6F8A866C
:1000E00051EC1BF001EE96F05AEC1BF0D00E9AEC9E
:1000F0001BF0000E9AEC1BF05AEC1BF0D10E9AECA0
:100100001BF00F9274EC1BF00F82EF6E69EC1BF08A
:10011000EFBEBFEF00F0BE0EA16FEF0EA26F5AEC64
:100120001BF0D00E9AEC1BF0010E9AEC1BF05AEC6F
:100130001BF0D10E9AEC1BF00F8274EC1BF0EC6EEE
:1001400074EC1BF0EC6E74EC1BF0EC6E74EC1BF0BA
:10015000EC6E74EC1BF0EC6E74EC1BF0EC6E0F921A
:1001600074EC1BF00F82EC6E69EC1BF0100EEF18B4
:10017000D8A4BFEF00F023EC12F004EF01F0010E61
:100180000627000E0723D8A0C9EF00F0FF0E066F68
:10019000076FDE0EA16FAD0EA26F2B6B2C6B2D6B5C
:1001A00001EE96F05AEC1BF0D00E9AEC1BF0000E0C
:1001B0009AEC1BF0000EEE6E9AEC1BF0000EEE6E49
:1001C0009AEC1BF0070EEE6E9AEC1BF0000EEE6E32
:1001D0009AEC1BF0070EEE6E9AEC1BF0040EEE6E1E
:1001E0009AEC1BF0210EEE6E9AEC1BF0100EEE6EE8
:1001F0009AEC1BF069EC1BF0FF0E146F166F176F73
:10020000000E156F186F196F8A9651EC1BF067EC92
:100210001CF07E800A0ED36E0F90F18AA56B010E42
:10022000AF6E000EB06E080EB86E260EAC6E900E5D
:10023000AB6E0E8C0EAC24EF01F0ACA21DEF01F002
:100240008B928B800A0EAD6EF2B289EC07F0F0B0A3
:10025000C9EC07F0F9EC1AF0FB6A020EFA6E2F31C6
:10026000E8303C0B6C0FD8B0FA2AF96E56EF01F06B
:10027000DFEF01F0EAEF03F060EF05F0B4EF05F017
:100280007AEF06F015EF07F08FEF08F064EF09F052
:1002900005EC1BF00EAC54EF01F0ACA24DEF01F0F9
:1002A0008B928B803F0EAD6E87EF07F00E80425130
:1002B000D8B466EF01F00E90E40E24EC1BF042512E
:1002C00024EC1BF0200EE3EC1AF0426B2E51D8B454
:1002D00075EF01F00E90D40E24EC1BF02E5124EC9F
:1002E0001BF0200EE3EC1AF02E6B0EA0DDEF01F0F8
:1002F0000EAAD8EF01F00E9A4C0E025DD8A490EF32
:1003000001F0370E035DD8A490EF01F0300E045DCC
:10031000D8A490EF01F0370E055DD8B49BEF01F043
:100320000E904C0E026F370E036F300E046F370EB7
:10033000056FD8EF01F00FB6A7EF01F0010EEFEC5B
:100340000EF08A0EC35C020EC458D8EF01F02A5199
:10035000D8B47AEF0AF0460E24EC1BF0080E2A5DA2
:10036000D8B4D3EF01F04C0E24EC1BF0080E2A5D3C
:10037000D8B4D3EF01F0550E24EC1BF0080E2A5D23
:10038000D8B4D3EF01F0530E24EC1BF0080E2A5D15
:10039000D8B4D3EF01F0480E24EC1BF0080E2A5D10
:1003A000D8A4CBEF01F0200EE3EC1AF0DDEF01F062
:1003B000FBEC07F00EA0DDEF01F087EF07F00EACCD
:1003C000E9EF01F0ACA2E2EF01F08B928B80440EDA
:1003D000AD6EFB6A030EFA6E3551A425E834E8349D
:1003E0003C0BEA0FD8B0FA2AF96E41EF02F04FEF5A
:1003F00002F055EF02F06FEF02F086EF02F0EEEF41
:1004000002F005EF03F055EF03F073EF03F091EF07
:1004100003F091EF03F091EF03F0B4EF03F0C8EFB6
:1004200003F0000000000000000005EC1BF00EAC23
:1004300021EF02F0ACA21AEF02F08B928B803F0EFC
:10044000AD6EDEEF03F0670EE96E000EEA6E3B5014
:10045000EE6E3C50EE6E3D50EE6E3E50EE6E3F50F6
:10046000EE6E1200670EE96E000EEA6EEE503B6E05
:10047000EE503C6EEE503D6EEE503E6EEE503F6ED6
:1004800012008B8ACD6AFD0ECF6E8F0ECE6E9E90BF
:10049000000ECC6E410ECD6E352BDEEF03F09EA02C
:1004A00053EF02F0352BDEEF03F0C4EC1BF0800EAF
:1004B0000BEC1CF0F30E0BEC1CF051EC1BF051ECB0
:1004C0001BF0D1EC1BF0100EA36FBA6A9D0EBB6E31
:1004D000BC6A9E92050EBA6E352BDEEF03F09EB21B
:1004E0007CEF02F03551D8A4A46F05EC1BF0100E80
:1004F000E3EC1AF084EF02F03551D8A483EF02F058
:10050000A451356FA46B352BDEEF03F03551A46F8A
:10051000C4EC1BF0810E0BEC1CF00FA4C1EF02F039
:10052000A3A996EF02F01D29D8A41D2BA3071E51E5
:10053000A35DA351D8A01E6FA351D8B4B4EF02F0AD
:10054000CD6AFF0ECF6E640ECE6E9E90000ECC6E06
:10055000410ECD6E05EC1BF0A46B030E356F100E33
:10056000E3EC1AF0D2EF02F08B9A51EC1BF005ECA1
:100570001BF0A46BAD0E206F216FDE0E226FD9EF42
:1005800003F00F82DEEC1BF0286F0F92DEEC1BF005
:10059000276F0F82D1EC1BF0A42B05EC1BF0100E83
:1005A000E3EC1AF0DEEF03F0C4EC1BF0800E0BEC72
:1005B0001CF0F30E0BEC1CF051EC1BF051EC1BF09B
:1005C000D1EC1BF0100EA36FBA6A9D0EBB6EBC6A15
:1005D0009E92050EBA6E352BDEEF03F09EB2FBEF56
:1005E00002F03551D8A4A46F05EC1BF0100EE3EC1B
:1005F0001AF003EF03F03551D8A402EF03F0A45131
:10060000356FA46B352BDEEF03F03551A46FC4ECCE
:100610001BF0810E0BEC1CF00FA442EF03F0D1ECA9
:100620001BF0A3A917EF03F01D29D8A41D2BA307C6
:100630001E51A35DA351D8A01E6FA351D8B435EFAE
:1006400003F0CD6AFF0ECF6E640ECE6E9E90000E4C
:10065000CC6E410ECD6E05EC1BF0A46B050E356F14
:10066000100EE3EC1AF053EF03F08B9A51EC1BF0F1
:1006700005EC1BF0A46BAD0E206F216FDE0E226F18
:10068000D9EF03F00F82DEEC1BF0256F0F92DEEC4A
:100690001BF0246F0F82D1EC1BF0A42B05EC1BF098
:1006A000100EE3EC1AF0DEEF03F027513B6E2851F9
:1006B0003C6E3D6A3E6A3F6AA40E406E440E416E37
:1006C000426A436A446A0CEC10F03B0E3D24216FF1
:1006D000010E3E20226FA42B05EC1BF0100EE3EC64
:1006E0001AF0DEEF03F02151165D22511759D8A000
:1006F0007EEF03F02151166F2251176F2151185DC3
:1007000022511959D8B089EF03F02151186F2251A5
:10071000196FA42B05EC1BF0100EE3EC1AF0DEEFC2
:1007200003F024513B6E25513C6E3D6A3E6A3F6AA0
:10073000E20E406E040E416E426A436A446A0CEC5B
:1007400010F0370E3D5C3B6E000E3E583C6E3D6A2D
:100750003E6A3F6A23EC02F0A42B05EC1BF0100E5E
:10076000E3EC1AF0DEEF03F032EC02F00A0E406E1A
:10077000416A426A436A446A3CEC10F03B50206F85
:10078000A42B05EC1BF0100EE3EC1AF0DEEF03F0E7
:100790002051145DD8A0CFEF03F02051146F2051E9
:1007A000155DD8B0D6EF03F02051156F05EC1BF0A6
:1007B000A46B700EE3EC1AF0DEEF03F00EACE8EF82
:1007C00003F0ACA2E1EF03F08B928B80640EAD6E70
:1007D00087EF07F00EACF4EF03F0ACA2EDEF03F0FF
:1007E0008B928B80580EAD6EFB6A080EFA6E0EACC3
:1007F00002EF04F0ACA2FAEF03F08B928B8035513C
:10080000300FAD6E3535E8341C0B120FD8B0FA2A14
:10081000F96E27EF04F031EF04F042EF04F048EFF7
:1008200004F0FAEF04F01FEF05F0000000000000F4
:10083000000005EC1BF00EAC25EF04F0ACA21EEF9F
:1008400004F08B928B803F0EAD6E54EF05F0352B8C
:10085000080E2A5DD8B02FEF04F005EC1BF054EF22
:1008600005F00E928BBA0E828B8ACD6AFD0ECF6E8A
:100870008F0ECE6E9E90000ECC6E410ECD6E352B3F
:1008800054EF05F09EA046EF04F0352B54EF05F031
:10089000070E0E15D8B457EF04F0080E0E27000E01
:1008A0000F23000E1023070EFF0A0E174289040EB5
:1008B000105DD8A061EF04F0060E105DD8A06BEFBC
:1008C00004F0000E0E6F1A6F000E0F6F1B6F040EF8
:1008D000106F1C6F428B040E1C5DD8A075EF04F0E6
:1008E000060E1C5DD8A07CEF04F00E511A6F0F515C
:1008F0001B6F10511C6F428D0E511A5D3B6E0F51D4
:100900001B593C6E10511C593D6ED8A0B1EF04F03C
:10091000D8B4B1EF04F03B1E3C1E3D1E010E3B2639
:10092000000E3C22000E3D22080E3B5CD8B0B1EF19
:1009300004F03C50D8A4B1EF04F03D50D8A4B1EF7E
:1009400004F0428F010E1B27000E1C23060E1C5DB7
:10095000D8A0B1EF04F0000E1A6F010E1B6F040E49
:100960001C6F040E0D5DD8A0BBEF04F0060E0D5DEC
:10097000D8A0C2EF04F00E510B6F0F510C6F105145
:100980000D6F428D0E510B5D3B6E0F510C593C6E3D
:1009900010510D593D6ED8A0F7EF04F0D8B4F7EF21
:1009A00004F03B1E3C1E3D1E010E3B26000E3C2269
:1009B000000E3D22080E3B5CD8B0F7EF04F03C502F
:1009C000D8A4F7EF04F03D50D8A4F7EF04F0428F1D
:1009D000010E0C27000E0D23060E0D5DD8A0B1EF01
:1009E00004F0000E0B6F010E0C6F040E0D6F352B13
:1009F00054EF05F0C4EC1BF010350E0BA0090BEC06
:100A00001CF00F510BEC1CF00E510BEC1CF0080EFF
:100A1000126E3BEC1BF00BEC1CF0122E09EF05F0F4
:100A2000D1EC1BF0CD6AFF0ECF6E380ECE6E9E90CD
:100A3000000ECC6E410ECD6E352B54EF05F09EA00E
:100A400052EF05F0080E0E27000E0F23000E1023A4
:100A5000060E105DD8A043EF05F0000E0E6F000EDD
:100A60000F6F040E106F0E511A5D0F511B5910516C
:100A70001C59D8A443EF05F0000E1A6F010E1B6F2E
:100A8000040E1C6F428F080E2A5DD8B050EF05F09F
:100A90000EA28B9A51EC1BF005EC1BF052EF05F007
:100AA000030E356F54EF05F00EAC5EEF05F0ACA20F
:100AB00057EF05F08B928B80780EAD6E87EF07F0C5
:100AC0000EAC6AEF05F0ACA263EF05F08B928B8061
:100AD0004E0EAD6EFB6A0A0EFA6E3535E8340C0B1D
:100AE000E80FD8B0FA2AF96E8AEF05F090EF05F01A
:100AF000A0EF05F00000000005EC1BF00EAC88EF45
:100B000005F0ACA281EF05F08B928B803F0EAD6EAD
:100B1000A8EF05F0A6B28EEF05F0352BA8EF05F093
:100B200005EC1BF005EC1BF0A96EF9EC1AF0DCECFF
:100B30000EF0020E356F300E1CEC1BF0A8EF05F026
:100B4000A6B2A6EF05F005EC1BF00E84A8EF05F0A9
:100B50000EACB2EF05F0ACA2ABEF05F08B928B8040
:100B60006E0EAD6E87EF07F00EACBEEF05F0ACA2D7
:100B7000B7EF05F08B928B80510EAD6EFB6A0B0EBA
:100B8000FA6E3535E8343C0B900FD8B0FA2AF96E7E
:100B9000F6EF05F003EF06F009EF06F020EF06F0A0
:100BA00041EF06F04AEF06F04FEF06F054EF06F083
:100BB00059EF06F0000000000000000000000000F7
:100BC0000000000000000000000000000000000025
:100BD00005EC1BF00EACF4EF05F0ACA2EDEF05F068
:100BE0008B928B803F0EAD6E6EEF06F0CD6AFF0EDE
:100BF000CF6EE00ECE6E9E90000ECC6E410ECD6E8E
:100C0000352B6EEF06F09EA007EF06F0352B6EEF4A
:100C100006F08A8651EC1BF05AEC1BF0D00E9AECD1
:100C20001BF0000E9AEC1BF05AEC1BF0D10E9AEC64
:100C30001BF00F8274EC1BF0C86F352B6EEF06F0C3
:100C4000010EEA6E970EE96E0F8274EC1BF0EE6EE9
:100C500074EC1BF0EE6E74EC1BF0EE6E74EC1BF09B
:100C6000EE6E74EC1BF0EE6E0F9274EC1BF00F82C4
:100C7000EE6E69EC1BF08A9651EC1BF0352B6EEF93
:100C800006F0FA0EA16FCE0EA26F67EC1CF0352BAA
:100C90006EEF06F02AEC12F0352B6EEF06F048EC02
:100CA00012F0352B6EEF06F060EC12F0352B6EEF84
:100CB00006F0FF0E146F166F176F000E156F186F8A
:100CC000196F100EE3EC1AF005EC1BF0500EE3EC7C
:100CD0001AF0600EE3EC1AF06EEF06F00EAC78EF4F
:100CE00006F0ACA271EF06F08B928B80710EAD6EA8
:100CF00087EF07F00EAC84EF06F0ACA27DEF06F0B4
:100D00008B928B80420EAD6E0EAC8EEF06F0ACA2D5
:100D100087EF06F08B928B804C0EAD6EFB6A0D0E4A
:100D2000FA6E3535E8340C0B300FD8B0FA2AF96E6C
:100D3000AEEF06F0BDEF06F0CDEF06F0FFEF06F0E8
:100D400005EC1BF00EACACEF06F0ACA2A5EF06F084
:100D50008B928B803F0EAD6E09EF07F08B928B80EC
:100D6000CD6AF30ECF6ECB0ECE6E9E90000ECC6E83
:100D7000410ECD6E352B09EF07F09EA0CBEF06F0AC
:100D8000010EC26E900EE8CF42FF42CFE8FFE8AC02
:100D9000C5EF06F0352B09EF07F0C282C2B2CEEFE5
:100DA00006F0C26A000EE8CF42FF8B908B828A0E5B
:100DB000C35C020EC458D8B0F2EF06F0C3503B6ECD
:100DC000C4503C6ED8903C323B32E10E3B5E000E8C
:100DD0003C5AD8A0F2EF06F03C50FF0ED8A43B6E70
:100DE0003B500A6FCD6AF30ECF6ECB0ECE6E9E9047
:100DF000000ECC6E410ECD6E352B09EF07F09EA094
:100E000007EF07F005EC1BF00F8607EF07F009EF7F
:100E100007F00EAC13EF07F0ACA20CEF07F08B92CB
:100E20008B80620EAD6E87EF07F00EAC1FEF07F000
:100E3000ACA218EF07F08B928B80530EAD6EF60EBE
:100E4000A66F24EC1BF0530EA62724EC1BF0530EC8
:100E5000A62724EC1BF0200EE16E010EE26EE65098
:100E6000A62724EC1BF0E650A62724EC1BF0E65046
:100E7000A62724EC1BF0E650AE51A62724EC1BF06D
:100E8000E650AF51A62724EC1BF0E650A62724EC31
:100E90001BF0E650A62724EC1BF0E6504C0EA627CC
:100EA00024EC1BF0E650370EA62724EC1BF0E6508E
:100EB000300EA62724EC1BF0E650370EA62724ECB4
:100EC0001BF0E650A62724EC1BF0E650A62724ECE6
:100ED0001BF0E650A62724EC1BF0E6500A51A6278B
:100EE00024EC1BF0A61D010F24EC1BF005EC1BF0FD
:100EF000200EE3EC1AF00EAC85EF07F0ACA27EEF0B
:100F000007F08B928B80730EAD6E87EF07F01AEFB0
:100F100001F0F2920EAC94EF07F0ACA28DEF07F067
:100F20008B928B80540EAD6E0E8A190E2B27D8A093
:100F3000A1EF07F0100EE3EC1AF0000E2C23000EC8
:100F40002D23800E2B5D510E2C59010E2D59D8A04A
:100F5000B2EF07F02B6B2C6B2D6B400EE3EC1AF00D
:100F6000C8EF07F0BB51BC11D8B4C0EF07F0010EB9
:100F7000BB5F000EBC5BBB51BC11D8A4C8EF07F02F
:100F8000600EE3EC1AF00F86B9C1BBF1BAC1BCF137
:100F900012000EACD3EF07F0ACA2CCEF07F08B92AF
:100FA0008B80520EAD6EF090010E1127000E1223B1
:100FB000000E1323D8A0E1EF07F0FF0E116F126FA0
:100FC000136F3E0E2A5D030FD8A0EBEF07F02E3D06
:100FD0002E2BFAEF07F02D51C60ED8A4C70E24EC25
:100FE0001BF02C5124EC1BF02B5124EC1BF0200E99
:100FF000E3EC1AF012000EAC05EF08F0ACA2FEEF25
:1010000007F08B928B80560EAD6E01EE02F01E0E35
:10101000126E000ED3EC0EF05A0AD8B415EF08F099
:10102000FF0AD8B418EF08F0FF00400E1BEF08F0DD
:10103000000E1BEF08F0A96EFB6A100EFA6EA535C4
:10104000E8340C0B4C0FD8B0FA2AF96E2EEF08F0EA
:1010500052EF08F06EEF08F080EF08F0020EA926BC
:10106000A69EA69CA680EE50A85CD8B447EF08F0D8
:10107000ED50EF50E16E300EE3EC1AF0A950E3ECC6
:101080001AF0E150E3EC1AF00E9084EF08F0A92A70
:10109000122E32EF08F00EA450EF08F0A52B0E90A0
:1010A00084EF08F0010EA924400AA96EA69EA69C12
:1010B000A680A850010FA86EFF0EA818D8B4A82AC1
:1010C000300EE3EC1AF0A950400AE3EC1AF0A850F5
:1010D000E3EC1AF0A52B0E9084EF08F0A950A50EB2
:1010E000D8B45A0EA86E300EE3EC1AF0000EE3EC02
:1010F0001AF0A850E3EC1AF0A52B0E9084EF08F03C
:101100000E94A56B84EF08F00EAC8EEF08F0ACA245
:1011100087EF08F08B928B80760EAD6E12000EACCE
:1011200099EF08F0ACA292EF08F08B928B80570EEB
:10113000AD6EFB6A110EFA6E3551E834E8343C0BA3
:10114000480FD8B0FA2AF96ECAEF08F0D8EF08F0C5
:10115000DEEF08F0000000000000000000000000CA
:10116000000000000000000000000000000000007F
:10117000000000000000000005EC1BF00EACC8EF02
:1011800008F0ACA2C1EF08F08B928B803F0EAD6EE1
:1011900058EF09F08B8ACD6AFD0ECF6E8F0ECE6EA2
:1011A0009E90000ECC6E410ECD6E352B58EF09F09F
:1011B0009EA0DCEF08F0352B58EF09F0800ED36EBF
:1011C0000F80B16AB36AB26AA192B46A040EE8CF22
:1011D00048FF030EB16E000EE8CF54FF7B94050E5E
:1011E000E8CF54FF7BB4FAEF08F0A1B245EF09F065
:1011F000F2EF08F07B9455CF55F056CF56F0040E21
:10120000E8CF54FF7BB40AEF09F0A1B245EF09F033
:1012100002EF09F07B9455CF57F056CF58F0050EEA
:10122000E8CF54FF7BB41AEF09F0A1B245EF09F003
:1012300012EF09F07B9455CF59F056CF5AF0000EBB
:10124000E8CF54FF5550575C3B6E565058583C6E93
:101250003D6A3E6A3F6A100E406E270E416E426A3A
:10126000436A446A0CEC10F05550595C406E56507D
:101270005A58416E426A436A446A3CEC10F03BC0E3
:10128000AEF13CC0AFF14CEF09F0B16A000EE8CF0F
:1012900054FFFF0EAE6FAF6F0A0ED36E0F9005ECCA
:1012A0001BF0040EB06F800EE3EC1AF058EF09F05B
:1012B0000EAC62EF09F0ACA25BEF09F08B928B8071
:1012C000770EAD6E87EF07F00EAC6EEF09F0ACA2B3
:1012D00067EF09F08B928B805A0EAD6E05EC1BF018
:1012E000B9EF09F0B16AB36AB26AB46AA192F1982F
:1012F000F092B06B010EB16EF0B287EF09F0A1A2CF
:101300007CEF09F0B03CB02BA1927CEF09F0B16A00
:10131000B36AB26A310EB16EF092F0B299EF09F091
:101320008DEF09F0B350800BD8A49CEF09F08DEF3E
:1013300009F0B16AA1EF09F0B16AB36AB26AA1EF2C
:1013400009F0B551B76FB651B86FB351B56FB4511D
:10135000B66FB151B36FB251B46FB250B16FB350F9
:10136000B26FB02FB9EF09F08B9A51EC1BF005EC7E
:101370001BF0C70ED56EEC0ED66EF294F2A4BEEF43
:1013800009F020C12EF02F6AFDEC0EF0ACA2C6EFE2
:1013900009F08B928B802C0EAD6EACA2CDEF09F0D4
:1013A0008B928B803350300FAD6EACA2D5EF09F02D
:1013B0008B928B803250300FAD6EACA2DDEF09F016
:1013C0008B928B803150300FAD6EC70ED56EEC0E08
:1013D000D66EF294F2A4EAEF09F021C12EF022C1F8
:1013E0002FF0FDEC0EF0ACA2F3EF09F08B928B80A6
:1013F0002C0EAD6EACA2FAEF09F08B928B803550BB
:10140000300FAD6EACA202EF0AF08B928B8034509D
:10141000300FAD6EACA20AEF0AF08B928B80335086
:10142000300FAD6EACA212EF0AF08B928B8032506F
:10143000300FAD6EACA21AEF0AF08B928B80315058
:10144000300FAD6EC70ED56EEC0ED66EF294F2A4D0
:1014500027EF0AF0AEC12EF0AFC12FF0FDEC0EF079
:10146000ACA230EF0AF08B928B802C0EAD6EACA24A
:1014700037EF0AF08B928B803550300FAD6EACA2F7
:101480003FEF0AF08B928B803450300FAD6EACA2E0
:1014900047EF0AF08B928B803350300FAD6EACA2C9
:1014A0004FEF0AF08B928B803250300FAD6EACA2B2
:1014B00057EF0AF08B928B803150300FAD6EACA29B
:1014C0005FEF0AF08B928B802C0EAD6E0EAC70EF3E
:1014D0000AF0ACA269EF0AF08B928B807A0EAD6EA7
:1014E000C70ED56E940ED66EF294F2A475EF0AF084
:1014F00087EF07F00FB665EF0CF07FEF0AF0F26AA6
:10150000800ED36E0F808B928B80470EAF6E000ED5
:10151000B06E080EB86E260EAC6E900EAB6E230E3B
:10152000756E000E766E080E706E260E726E980E38
:10153000CF68CE68810ECD6E160EBB6EBC6A3E0EB5
:10154000BA6E020EE8CF4BFF000EE8CF4CFF3E0E06
:10155000E8CF4AFF010EE8CF49FFFF0EE8500C0E1E
:10156000BD6E110EB96E000EBE6E060EE8CF51FFB5
:101570003F0E636F646F7F0E656F666F766B9F6A59
:10158000A26AA56A7C6A7F6A9D829F8A9D8A7F84FF
:101590007D84406B416B426B050E486F640E466F55
:1015A000C40E476F946B956BD08EF28CF28E0C94B8
:1015B0000C966DEC1FF0DDEF0AF083EC0DF0D8B067
:1015C000D2EC1CF0F2A2E9EF0AF0F2920E8ADDEF03
:1015D0000AF00EAAF7EF0AF00E9A010EEFEC0EF0E9
:1015E0008A0EC35C020EC458D8A0C7EF0CF0DDEF22
:1015F0000AF075EF0EF085EF0EF0415400004154F3
:101600004530000041542B4353434C4B3D310000C7
:1016100041542B434D47463D3100000041542B437C
:101620005245473F000041542B434D47533D220054
:1016300000002B323738323531303537383222001E
:101640000000436C65616E20737769746368204C99
:1016500031323600000041542B434D474C3D22416E
:101660004C4C2200000041542B434D47533D000099
:1016700041542B434D47443D000041542B435351AB
:10168000000041542B43474154543F000000415453
:101690002B53415042523D332C312C22434F4E5458
:1016A000595045222C2247505253220000004154E9
:1016B0002B53415042523D332C312C2241504E226B
:1016C0002C22494E5445524E4554220000004154AC
:1016D0002B53415042523D312C31000041542B5389
:1016E000415042523D322C31000041542B48545459
:1016F00050494E495400000041542B485454505016
:101700004152413D22434944222C310000004154C2
:101710002B48545450504152413D2255524C222C9A
:1017200022687474703A2F2F6661726D696E672E2D
:101730006167726967656C2E636F2E7A612F696EBF
:101740006465782F6170692F6170695F646174618D
:101750002E7068702200000041542B4854545050A1
:101760004152413D22434F4E54454E54222C22615A
:1017700070706C69636174696F6E2F782D777777FD
:101780002D666F726D2D75726C656E636F64656426
:101790002200000041542B48545450444154413DD0
:1017A00000002C313030303000006E616D653D61DD
:1017B0006A61785F70696E6700006E616D653D7289
:1017C0006426646174613D33413831000000304467
:1017D000000041542B48545450414354494F4E3D0E
:1017E0003100000041542B485454505245414400AC
:1017F000000041542B485454505445524D000000B1
:1018000041542B53415042523D302C3100004F4B3C
:101810000000415400004154453000004552524FF1
:10182000520000002B435245473A20302C31000033
:101830002B435245473A20302C35000041542B436E
:1018400050494E3F00002B4350494E3A20524541EB
:10185000445900002B4350494E3A2053494D2050E3
:10186000494E00002B435343413A00002B434D4760
:10187000533A00002B434D474C3A00002B4347415D
:1018800054543A20310000002B53415042523A0048
:101890000000444F574E4C4F414400002B485454D5
:1018A00050414354494F4E3A00002B485454505233
:1018B0004541443A00002B485454505445524D0081
:1018C00000002B4353513A000000F26A800ED36EA1
:1018D0000F808B908B82170EAF6E000EB06E080ECD
:1018E000B86E260EAC6E900EAB6E230E756E000EAB
:1018F000766E080E706E260E726E980ECF68CE68E9
:10190000810ECD6E160EBB6EBC6A3E0EBA6E020E16
:10191000E8CF4BFF000EE8CF4CFF3E0EE8CF4AFF6A
:10192000010EE8CF49FFFF0EE8500C0EBD6E110E00
:10193000B96E000EBE6E060EE8CF51FF3F0E636F0C
:10194000646F7F0E656F666F766B9F6AA26AA56A89
:101950007C6A7F6A9D829F8A9D8A7F847D84406B9A
:10196000416B426B050E486F640E466FC40E476FA5
:10197000946B956BD08EF28CF28E000E916F6DECA5
:1019800012F091C1E8FF580AD8A4BFEF0CF0F26A38
:101990008B908B820CA4D8EF0CF00C94010E0827CE
:1019A000000E0923D8A0D8EF0CF0FF0E086F096FC6
:1019B0006DEC1FF08A8651EC1BF001EE96F05AECAC
:1019C0001BF0D00E9AEC1BF0000E9AEC1BF05AECB8
:1019D0001BF0D10E9AEC1BF00F8274EC1BF0EE6E34
:1019E00074EC1BF0EE6E74EC1BF0EE6E74EC1BF0FE
:1019F000EE6E74EC1BF0EE6E74EC1BF0EE6E74EC9D
:101A00001BF0EE6E0F9274EC1BF00F82EF6E69EC20
:101A10001BF0100EEF18D8B41BEF0DF05AEC1BF0B2
:101A2000D00E9AEC1BF0070E9AEC1BF0100E9AECFD
:101A30001BF069EC1BF08A9623EC12F00CA628EF41
:101A40000DF00C96FE0EA16FED0EA26F67EC1CF070
:101A50000A0ED36E0F901AEF01F06C6F6C390F0BFA
:101A6000300F832767EC0DF06C510F0B300F83277D
:101A700067EC0DF01200FDEC0EF03550300F8327AF
:101A800067EC0DF03450300F832767EC0DF03350C6
:101A9000300F832767EC0DF03250300F832767EC4F
:101AA0000DF03150300F832767EC0DF012002C0E33
:101AB000832767EC0DF012000A0E832767EC0DF008
:101AC0000D0E832767EC0DF01200BFEF0CF01C6EBB
:101AD00022EE40F06629800AD8B4C00E800AD96E82
:101AE000D9506519D8B470EF0DF01C50DF6ED95085
:101AF000666F1C501200F29EF2BE7BEF0DF064C1C7
:101B000063F1F28E120063516419D8A4D880D8B45E
:101B1000D890D8B49EEF0DF093EF0DF06351641997
:101B2000D8B48EEF0DF022EE00F06329400AD8B44D
:101B3000400E400AD96E636FDF50D880120022EE4B
:101B400040F065516619D8B4AFEF0DF06529800AF1
:101B5000D8B4C00E800AD96E656FDF50AD6E12002A
:101B60000890ABA2BDEF0DF00880AB98ABB8B5EF15
:101B70000DF0AB88ABA8B9EF0DF0ABA4C2EF0DF040
:101B80000880AE5008B0D9EF0DF022EE00F06429C5
:101B9000400AD8B4400E400AD96E6319D8B4D7EFC2
:101BA0000DF0AE50DF6ED950646FD9EF0DF0AE502E
:101BB00008821200D00E8CEC10F0000E8CEC10F0AD
:101BC00025508CEC10F026508CEC10F027508CEC4B
:101BD00010F028508CEC10F029508CEC10F02A50AA
:101BE0008CEC10F02B508CEC10F02C508CEC10F096
:101BF0001200D00E8CEC10F0000E8CEC10F0D10E18
:101C00008CEC10F08CEC10F0256E8CEC10F0266E45
:101C10008CEC10F0276E8CEC10F0286E8CEC10F031
:101C2000296E8CEC10F02A6E8CEC10F02B6E8CEC84
:101C300010F02C6E120030EC0EF030EC0EF030ECA8
:101C40000EF030EC0EF030EC0EF030EC0EF030EC2C
:101C50000EF030EC0EF030EC0EF030EC0EF0120026
:101C600045EC0EF045EC0EF045EC0EF045EC0EF0B8
:101C700045EC0EF045EC0EF045EC0EF045EC0EF0A8
:101C800045EC0EF045EC0EF012005AEC0EF05AEC5A
:101C90000EF05AEC0EF05AEC0EF05AEC0EF05AEC34
:101CA0000EF05AEC0EF05AEC0EF05AEC0EF05AEC24
:101CB0000EF01200C70ED56E940ED66EF294F2A4FA
:101CC0005FEF0EF01200C70ED56EF50ED66EF294D1
:101CD000F2A468EF0EF01200C70ED56EFA0ED66EA3
:101CE000F294F2A471EF0EF01200D9CF3EF1DACFE8
:101CF0003FF19EBAB0EC0DF0ACB29FEC0DF07E94CB
:101D00003FC1DAFF3EC1D9FF1100E8CF36F1D8CF8D
:101D100037F1E2CF39F1E1CF38F1DACF3BF1D9CF6A
:101D20003AF1FACF3CF1FBCF3DF19EB2A9EC0EF0B7
:101D300036C1E8FF37C1D8FF39C1E2FF38C1E1FF42
:101D40003BC1DAFF3AC1D9FF3CC1FAFF3DC1FBFFFD
:101D50001000C282482FD1EF0EF0050E486F0A8E98
:101D600094519511D8B4BDEF0EF0010E945F000EA2
:101D7000955B94519511D8B4408DC282462FC4EF23
:101D80000EF0640E466F087E472FD1EF0EF0C40EA2
:101D9000476F5D51D8A4D0EF0EF00A82D1EF0EF05C
:101DA0005D079E921200A6B2D3EF0EF0A96EA69E1A
:101DB000A69CA680A8501200A6B2DCEF0EF0A86E7A
:101DC000A69EA69CA684F29EF2BEE3EF0EF0550EF0
:101DD000A76EAA0EA76EA682F28EA6941200C26EFD
:101DE000A00EE8CF42FF42CFE8FFE8ACF3EF0EF0E1
:101DF000C282C2B2F9EF0EF01200316A326A336A5F
:101E0000346A356A100E2E5E270E2F5AD8A00CEFBA
:101E10000FF0352A02EF0FF0100E2E26270E2F227C
:101E2000E80E2E5E030E2F5AD8A01AEF0FF0342AB8
:101E300010EF0FF0E80E2E26030E2F22640E2E5EFA
:101E4000000E2F5AD8A028EF0FF0332A1EEF0FF004
:101E5000640E2E26000E2F220A0E2E5ED8A034EF1E
:101E60000FF0322A2CEF0FF00A0E2E24316E1200E2
:101E7000316A326A336A346A356A366A376A386A6E
:101E8000800E2E5E960E2F5A980E305AD8A04CEF28
:101E90000FF0382A40EF0FF0800E2E26960E2F22DC
:101EA000980E3022400E2E5E420E2F5A0F0E305AE0
:101EB000D8A05EEF0FF0372A52EF0FF0400E2E261B
:101EC000420E2F220F0E3022A00E2E5E860E2F5AAB
:101ED000010E305AD8A070EF0FF0362A64EF0FF0E1
:101EE000A00E2E26860E2F22010E3022100E2E5E00
:101EF000270E2F5A000E305AD8A082EF0FF0352A45
:101F000076EF0FF0100E2E26270E2F22E80E2E5EF3
:101F1000030E2F5AD8A090EF0FF0342A86EF0FF05F
:101F2000E80E2E26030E2F22640E2E5E000E2F5A70
:101F3000D8A09EEF0FF0332A94EF0FF0640E2E26F8
:101F4000000E2F220A0E2E5ED8A0AAEF0FF0322A22
:101F5000A2EF0FF00A0E2E24316E120040503B26E5
:101F6000000ED8B0010E3C263994D8B039844150C7
:101F70003C26D8B03984000E39B4010E3D26399480
:101F8000D8B0398442503D26D8B03984000E39B4D7
:101F9000010E3E263994D8B0398443503E26D8B03D
:101FA0003984000E39B4010E3F263994D8B03984F3
:101FB00044503F2639B4D880120040503B5E000E9A
:101FC000D8A0010E3C5E3984D8A0399441503C5EC3
:101FD000D8A03994000E39A4010E3D5E3984D8A0F2
:101FE000399442503D5ED8A03994000E39A4010EB8
:101FF0003E5E3984D8A0399443503E5ED8A03994CF
:10200000000E39A4010E3F5E3984D8A039944450A3
:102010003F5E39A4D8901200399239963BC045F002
:102020003CC046F03DC047F03EC048F03FC049F0DC
:102030003B6A3C6A3D6A3E6A3F6A280E3A6E493204
:102040004832473246324532398439A63994D8A0CD
:10205000399439B43982D8B0AEEC0FF0D8B03982A7
:10206000D89040364136423643364436D8B0398669
:102070003A2E1FEF10F012003992405041104210DA
:1020800043104410D8B439823BC045F03CC046F000
:102090003DC047F03EC048F03FC049F03B6A3C6A53
:1020A0003D6A3E6A3F6A280E3A6E453646364736E6
:1020B000483649363B363C363D363E363F36DDEC1B
:1020C0000FF03988D8A03998D8A0AEEC0FF0D8809E
:1020D00039A8D8903A2E55EF10F045364636473697
:1020E0004836493645C03BF046C03CF047C03DF05D
:1020F00048C03EF049C03FF012003B380F0B3C6E29
:102100000F0E3B163C50D8B48BEF10F00A0E3B2656
:102110003C0682EF10F0120012004091800E4D6ECE
:10212000000E4C6E120083EC0DF0D8A0DBEF10F027
:102130004E6E4D50D8B4B0EF10F024EE00F04C507D
:10214000D96E4C2A4E50DF6E4D060D0AD8B4B0EF52
:1021500010F0070AD8B4B0EF10F093EF10F04083FE
:1021600024EE00F0800E4F6E4D504F5E4F2EBDEFAF
:1021700010F08DEC10F093EF10F0DF504095DCEC98
:1021800010F040A5C8EF10F08DEC10F093EF10F0B8
:10219000F4EC10F0A68EF86A180EF76E0E0EF66EBE
:1021A000130E546E31EC11F0D8B0D9EF10F0FF0ED1
:1021B000526E52504081120040B5EFEF10F0DF50E8
:1021C000200AD8B4EAEF10F0290AD8B4EAEF10F0E8
:1021D000EFEF10F0D92A4F2EDCEF10F04085D950E8
:1021E000506E516ADF50120040B502EF11F080ECE2
:1021F00011F0D8A002EF11F0D92A512A4F2EF4EF96
:1022000010F04085DF505152120040B513EF11F02D
:10221000D7EC11F0D8A013EF11F0D92A512A4F2E84
:1022200005EF11F04085DF505152120040B524EF08
:1022300011F0FDEC11F0D8A024EF11F0D92A512AA9
:102240004F2E16EF11F04085DF505152120040B56D
:102250002FEF11F0D92A4F2E2FEF11F04085DF50CC
:1022600012005150D8B45FEF11F0526A5050D96E3D
:102270005150536E0900F550FF0BD8B454EF11F0D4
:10228000DF5CD8A44EEF11F0D92A532E3AEF11F0AB
:102290000900F550FF0BD8B462EF11F00900F550BA
:1022A000FF0BD8A44EEF11F00900F550FF0BD8B486
:1022B00054EF11F00A00522A542E36EF11F0D89044
:1022C00063EF11F0D8801200410EDF5CD8A07DEFE3
:1022D00011F05B0EDF5CD8A07AEF11F0610EDF5CCD
:1022E000D8A07DEF11F07B0EDF5CD8B07DEF11F050
:1022F000200EDF5ED8807EEF11F0D890DF50120004
:10230000200EDF5C40ABD894D8B4D1EF11F0210E91
:10231000DF5CD8B4D1EF11F0220E40A9230EDF5CB0
:10232000D8A0D4EF11F02C0EDF5CD8A0D1EF11F0C3
:102330002C0E40AB2D0EDF5CD8A0D4EF11F0300E88
:10234000DF5CD8A0D1EF11F0300EDF5CD8A0D4EF65
:1023500011F03A0EDF5CD8A0D1EF11F03A0EDF5C3D
:10236000D8A0D4EF11F0410EDF5CD8A0D1EF11F06E
:10237000410EDF5CD8A0D4EF11F05B0EDF5CD8A07B
:10238000D1EF11F0610EDF5CD8A0D4EF11F07B0E1D
:10239000DF5CD8B0D4EF11F040A7D1EF11F0200EE0
:1023A000DF5ED880D5EF11F0D890DF501200300EEC
:1023B000DF5CD8A0FAEF11F03A0EDF5CD8A0F7EF9F
:1023C00011F0410EDF5CD8A0FAEF11F05B0EDF5C7C
:1023D000D8A0F7EF11F0610EDF5CD8A0FAEF11F092
:1023E0007B0EDF5CD8B0FAEF11F0200EDF5ED880F4
:1023F000FBEF11F0D890DF501200300EDF5CD8A058
:102400000AEF12F03A0EDF5CD8B00AEF12F0D88073
:102410000BEF12F0D890DF501200906F903919EC4A
:1024200012F067EC0DF0905119EC12F067EC0DF022
:1024300012000F0B300F8F6F3A0E8F5D070ED8A072
:10244000000E8F2512002AEC12F048EC12F060EC1E
:1024500012F0120098513B6E7DEC10F0070E3B5CC1
:10246000F90ED8A0110E3B263C6A3D6A3E6A3F6ACF
:10247000100E406E0E0E416E426A436A446A0CECC6
:1024800010F03B502B6F3C502C6F3D502D6F1200C5
:1024900097513B6E7DEC10F03C6A3D6A3E6A3F6AA4
:1024A0003C0E406E000E416E426A436A446A0CEC78
:1024B00010F03B502B273C502C233D502D23120075
:1024C00096513B6E7DEC10F03C6A3D6A3B502B27E9
:1024D0003C502C233D502D231200FB6A91C192F1F8
:1024E000936BD8909237933792379337FA0E92279F
:1024F000240E9321FA6E9251F96E3DEF13F042EFE4
:1025000013F047EF13F05BEF13F066EF13F06EEF8D
:1025100013F075EF13F08CEF13F0A0EF13F0BDEF95
:1025200013F0CCEF13F0E5EF13F0F8EF13F013EF27
:1025300014F01AEF14F033EF14F046EF14F055EFE7
:1025400014F05CEF14F073EF14F086EF14F095EFD5
:1025500014F09CEF14F0B3EF14F0C6EF14F0D5EFC5
:1025600014F0DCEF14F0F3EF14F006EF15F022EFA7
:1025700015F029EF15F040EF15F053EF15F064EF6B
:1025800015F06BEF15F082EF15F095EF15F0A6EF53
:1025900015F0ADEF15F0C4EF15F0D7EF15F0E8EF3B
:1025A00015F0EFEF15F006EF16F019EF16F035EF16
:1025B00016F03CEF16F053EF16F066EF16F077EFDB
:1025C00016F07EEF16F095EF16F0A8EF16F0B9EFC3
:1025D00016F0C0EF16F0D7EF16F0EAEF16F0FBEFAB
:1025E00016F002EF17F019EF17F02CEF17F03DEF90
:1025F00017F044EF17F0AFEF17F0C2EF17F0D3EF7B
:1026000017F0DAEF17F040EF18F053EF18F065EF1E
:1026100018F06CEF18F083EF18F096EF18F0B5EFA4
:1026200018F0BCEF18F0D3EF18F0E6EF18F01EEF3B
:1026300019F025EF19F03CEF19F04FEF19F060EFAA
:1026400019F067EF19F07EEF19F091EF19F043EFF1
:102650001AF05FEF1AF06AEF1AF07CEF1AF07EEFD3
:102660001AF0A3EF19F0AAEF19F0D1EF19F0EFEF7C
:1026700019F015EF1AF028EF1AF0010EE8CF91F1DA
:102680006DEF12F0020EE8CF91F186EF1AF0899605
:1026900080B453EF13F0898A87EC1AF0030EE8CF69
:1026A00091F186EF1AF0899AABEC1AF0040EE8CF9C
:1026B00091F186EF1AF040AD64EF13F0899AABEC1C
:1026C0001AF0040EE8CF91F186EF1AF040AD6CEFEE
:1026D00013F0050EE8CF91F186EF1AF099EC1AF09D
:1026E000060EE8CF91F186EF1AF040AD8AEF13F0B5
:1026F0007BEC0DF0409FA68EF86A150EF76EFA0E71
:10270000F66ECCEC1AF09FEC1AF08DEC10F0070E80
:10271000E8CF91F186EF1AF0408B93EC10F040A1D6
:1027200097EF13F0080EE8CF91F16DEF12F040AD86
:102730009EEF13F04191000EE8CF91F186EF1AF071
:102740005250010AD8A4ADEF13F041838DEC10F084
:10275000070EE8CF91F16DEF12F0010AD8A4B7EFA0
:1027600013F04181090EE8CF91F1BBEF13F04191D5
:10277000000EE8CF91F186EF1AF041B3C5EF13F0E8
:102780000D0EE8CF91F1CAEF13F099EC1AF00A0E92
:10279000E8CF91F186EF1AF040ADE3EF13F07BEC58
:1027A0000DF0409FA68EF86A150EF76EFE0EF66EBF
:1027B000CCEC1AF09FEC1AF08DEC10F00B0EE8CF79
:1027C00091F16DEF12F086EF1AF0408B93EC10F060
:1027D00040A1F0EF13F00C0EE8CF91F16DEF12F085
:1027E00040ADF6EF13F0000EE8CF91F186EF1AF04E
:1027F0005250020AD8A404EF14F08DEC10F00B0E26
:10280000E8CF91F16DEF12F0020AD8A40EEF14F0A8
:1028100041930D0EE8CF91F111EF14F0000EE8CFC7
:1028200091F186EF1AF099EC1AF00E0EE8CF91F1C3
:1028300086EF1AF040AD31EF14F07BEC0DF0409FC5
:10284000A68EF86A160EF76E040EF66ECCEC1AF031
:102850009FEC1AF08DEC10F00F0EE8CF91F16DEFB8
:1028600012F086EF1AF0408B93EC10F040A13EEF8F
:1028700014F0100EE8CF91F16DEF12F040AD44EF7F
:1028800014F0000EE8CF91F186EF1AF05250000AD2
:10289000D8A450EF14F0110EE8CF91F16DEF12F0C3
:1028A000550EE8CF91F186EF1AF099EC1AF0120E5E
:1028B000E8CF91F186EF1AF040AD71EF14F07BECA8
:1028C0000DF0409FA68EF86A160EF76E100EF66E8B
:1028D000CCEC1AF09FEC1AF08DEC10F0130EE8CF50
:1028E00091F186EF1AF0408B93EC10F040A17EEF4F
:1028F00014F0140EE8CF91F16DEF12F040AD84EFBB
:1029000014F0000EE8CF91F186EF1AF05250000A51
:10291000D8A490EF14F0150EE8CF91F193EF14F0D6
:10292000000EE8CF91F186EF1AF099EC1AF0160E2E
:10293000E8CF91F186EF1AF040ADB1EF14F07BECE7
:102940000DF0409FA68EF86A160EF76E1C0EF66EFE
:10295000CCEC1AF09FEC1AF08DEC10F0170EE8CFCB
:1029600091F186EF1AF0408B93EC10F040A1BEEF8E
:1029700014F0180EE8CF91F16DEF12F040ADC4EFF6
:1029800014F0550EE8CF91F186EF1AF05250040A78
:10299000D8A4D0EF14F01D0EE8CF91F1D3EF14F0CE
:1029A000150EE8CF91F186EF1AF099EC1AF01A0E95
:1029B000E8CF91F186EF1AF040ADF1EF14F07BEC27
:1029C0000DF0409FA68EF86A160EF76E820EF66E18
:1029D000CCEC1AF0B6EC1AF08DEC10F01B0EE8CF30
:1029E00091F186EF1AF0408B93EC10F040A1FEEFCE
:1029F00014F01C0EE8CF91F16DEF12F040AD04EF32
:102A000015F0550EE8CF91F186EF1AF052500C0AEE
:102A1000D8A4D0EF14F08DEC10F01B0EE8CF91F19C
:102A200020EF15F00C0AD8A41BEF15F01D0EE8CF0F
:102A300091F120EF15F0550EE8CF91F120EF15F050
:102A400086EF1AF099EC1AF01E0EE8CF91F186EF9E
:102A50001AF040AD3EEF15F07BEC0DF0409FA68ED6
:102A6000F86A160EF76E8E0EF66ECCEC1AF09FEC2E
:102A70001AF08DEC10F01F0EE8CF91F186EF1AF0EE
:102A8000408B93EC10F040A14BEF15F0200EE8CFF7
:102A900091F16DEF12F040AD51EF15F0550EE8CF0A
:102AA00091F186EF1AF05250000AD8A45DEF15F0AC
:102AB000210EE8CF91F120EF15F0550EE8CF91F1FE
:102AC00062EF15F086EF1AF08DEC1AF0220EE8CFC7
:102AD00091F186EF1AF040AD80EF15F07BEC0DF030
:102AE000409FA68EF86A160EF76EAE0EF66ECCEC10
:102AF0001AF09FEC1AF08DEC10F0230EE8CF91F154
:102B000086EF1AF0408B93EC10F040A18DEF15F09A
:102B1000240EE8CF91F16DEF12F040AD93EF15F078
:102B2000550EE8CF91F186EF1AF05250000AD8A462
:102B30009FEF15F0250EE8CF91F1A4EF15F0550E9B
:102B4000E8CF91F1A4EF15F086EF1AF08DEC1AF0B2
:102B5000260EE8CF91F186EF1AF040ADC2EF15F0E6
:102B60007BEC0DF0409FA68EF86A160EF76ECE0E27
:102B7000F66ECCEC1AF0C1EC1AF08DEC10F0270ECA
:102B8000E8CF91F186EF1AF0408B93EC10F040A162
:102B9000CFEF15F0280EE8CF91F16DEF12F040ADB8
:102BA000D5EF15F0550EE8CF91F186EF1AF052509F
:102BB000000AD8A4E1EF15F0290EE8CF91F1E6EF75
:102BC00015F0550EE8CF91F1E6EF15F086EF1AF00B
:102BD0008DEC1AF02A0EE8CF91F186EF1AF040AD95
:102BE00004EF16F07BEC0DF0409FA68EF86A160EEF
:102BF000F76EDC0EF66ECCEC1AF0C1EC1AF08DEC30
:102C000010F02B0EE8CF91F186EF1AF0409B93EC79
:102C100010F040A111EF16F02C0EE8CF91F16DEFFE
:102C200012F040AD17EF16F0550EE8CF91F186EF98
:102C30001AF052500D0AD8A425EF16F08DEC10F0C2
:102C40002B0EE8CF91F120EF15F00D0AD8A42EEF4E
:102C500016F02D0EE8CF91F133EF16F0550EE8CFB8
:102C600091F133EF16F086EF1AF08DEC1AF02E0E7C
:102C7000E8CF91F186EF1AF040AD51EF16F07BEC02
:102C80000DF0409FA68EF86A160EF76EEA0EF66EED
:102C9000CCEC1AF09FEC1AF08DEC10F02F0EE8CF70
:102CA00091F186EF1AF0408B93EC10F040A15EEFAB
:102CB00016F0300EE8CF91F16DEF12F040AD64EFF9
:102CC00016F0550EE8CF91F186EF1AF05250000A37
:102CD000D8A470EF16F0310EE8CF91F175EF16F031
:102CE000550EE8CF91F175EF16F086EF1AF08DECE6
:102CF0001AF0320EE8CF91F186EF1AF040AD93EF63
:102D000016F07BEC0DF0409FA68EF86A160EF76E5B
:102D1000F80EF66ECCEC1AF09FEC1AF08DEC10F079
:102D2000330EE8CF91F186EF1AF0408B93EC10F060
:102D300040A1A0EF16F0340EE8CF91F16DEF12F044
:102D400040ADA6EF16F0550EE8CF91F186EF1AF0E0
:102D50005250000AD8A4B2EF16F0350EE8CF91F128
:102D6000B7EF16F0550EE8CF91F1B7EF16F086EFFA
:102D70001AF08DEC1AF0360EE8CF91F186EF1AF0CA
:102D800040ADD5EF16F07BEC0DF0409FA68EF86AB3
:102D9000170EF76E0E0EF66ECCEC1AF09FEC1AF0D2
:102DA0008DEC10F0370EE8CF91F186EF1AF0408BE2
:102DB00093EC10F040A1E2EF16F0380EE8CF91F15D
:102DC0006DEF12F040ADE8EF16F0550EE8CF91F13F
:102DD00086EF1AF05250000AD8A4F4EF16F0390E1C
:102DE000E8CF91F1A4EF15F0550EE8CF91F1F9EF8E
:102DF00016F086EF1AF08DEC1AF03A0EE8CF91F14A
:102E000086EF1AF040AD17EF17F07BEC0DF0409F06
:102E1000A68EF86A170EF76E580EF66ECCEC1AF006
:102E20009FEC1AF08DEC10F03B0EE8CF91F186EF9D
:102E30001AF0408B93EC10F040A124EF17F03C0EF9
:102E4000E8CF91F16DEF12F040AD2AEF17F0550E7B
:102E5000E8CF91F186EF1AF05250000AD8A436EF6D
:102E600017F03D0EE8CF91F13BEF17F0550EE8CF8C
:102E700091F13BEF17F086EF1AF08DEC1AF03E0E51
:102E8000E8CF91F186EF1AF040ADADEF17F07BEC93
:102E90000DF01A510E5D3B6E1B510F593C6E1C51CB
:102EA00010593D6ED8B061EF17F0000E3B6E000E6A
:102EB0003C6E060E3D6E1A513B5E1B513C5A1C5136
:102EC0003D5AFC0E3B5C000E3C58000E3D58FB0E7C
:102ED000D8B03B6E3B50A76F040E3B263B50A86F0B
:102EE000BB0EA96F3C6AD8903B363C36170E3B268A
:102EF000000E3C223BC02EF03CC02FF0FDEC0EF04B
:102F0000408FA68EF86A170EF76E940EF66ECCEC14
:102F10001AF0300E352467EC0DF0300E342467ECD7
:102F20000DF0300E332467EC0DF0300E322467ECD8
:102F30000DF0300E312467EC0DF0409FA68EF86A3C
:102F4000170EF76EA20EF66ECCEC1AF09FEC1AF08C
:102F50008DEC10F03F0EE8CF91F186EF1AF0408B28
:102F600093EC10F040A1BAEF17F0400EE8CF91F1CA
:102F70006DEF12F040ADC0EF17F0550EE8CF91F1B4
:102F800086EF1AF052500E0AD8A4CCEF17F0410E7B
:102F9000E8CF91F1D1EF17F0550EE8CF91F1D1EFD5
:102FA00017F086EF1AF08DEC1AF0420EE8CF91F18F
:102FB00086EF1AF040AD3EEF18F07BEC0DF0408F3D
:102FC000A68EF86A170EF76EBA0EF66ECCEC1AF0F3
:102FD000A851A9270DEC12F0800ED3EC0EF0A92712
:102FE0000DEC12F0810ED3EC0EF0A9270DEC12F0CF
:102FF000820ED3EC0EF0A9270DEC12F0830ED3EC69
:103000000EF0A9270DEC12F0040EA85FD8B42BEF38
:1030100018F01AC11EF01BC11FF01CC120F08B8AD2
:1030200063EC0EF0C4EC1BF020340E0BA0090BEC8B
:103030001CF01F500BEC1CF01E500BEC1CF037EC7E
:103040001CF04FEC1CF0A9270DEC12F0A82F21EF7B
:1030500018F055EC1CF0A91D0DEC12F0409FA68E47
:10306000F86A170EF76ECE0EF66ECCEC1AF09FECE7
:103070001AF08DEC10F0430EE8CF91F186EF1AF0C4
:10308000408B93EC10F040A14BEF18F0440EE8CFCA
:1030900091F16DEF12F040AD51EF18F0550EE8CF01
:1030A00091F186EF1AF08B9A5250000AD8A45EEF85
:1030B00018F0450EE8CF91F1D1EF17F0550EE8CF9B
:1030C00091F163EF18F086EF1AF08DEC1AF0460ECE
:1030D000E8CF91F186EF1AF040AD81EF18F07BEC6C
:1030E0000DF0409FA68EF86A170EF76ED20EF66EA0
:1030F000CCEC1AF09FEC1AF08DEC10F0470EE8CFF4
:1031000091F186EF1AF0409B93EC10F040A18EEF06
:1031100018F0480EE8CF91F16DEF12F040AD94EF4A
:1031200018F0550EE8CF91F186EF1AF052500F0AC1
:10313000D8A4A0EF18F0490EE8CF91F1B3EF18F042
:103140005250000AD8A4AEEF18F09FEC1AF08DECA4
:1031500010F0470EE8CF91F1B3EF18F0550EE8CF1D
:1031600091F1B3EF18F086EF1AF099EC1AF04A0ECD
:10317000E8CF91F186EF1AF040ADD1EF18F07BEC7B
:103180000DF0409FA68EF86A170EF76EE40EF66EED
:10319000CCEC1AF09FEC1AF08DEC10F04B0EE8CF4F
:1031A00091F186EF1AF0409B93EC10F040A1DEEF16
:1031B00018F04C0EE8CF91F16DEF12F040ADE4EF56
:1031C00018F0550EE8CF91F186EF1AF05250100A20
:1031D000D8A417EF19F0A7511A27000E1B23000ED1
:1031E0001C23060E1C5DD8A0FCEF18F0000E1A6F11
:1031F000000E1B6F040E1C6F1A510E19D8A410EF8D
:1032000019F01B510F19D8A410EF19F01C51101907
:10321000D8A4FCEF18F04D0EE8CF91F115EF19F09E
:103220003D0EE8CF91F115EF19F01CEF19F0550E96
:10323000E8CF91F11CEF19F086EF1AF099EC1AF033
:103240004E0EE8CF91F186EF1AF040AD3AEF19F04B
:103250007BEC0DF0409FA68EF86A170EF76EF20E0B
:10326000F66ECCEC1AF09FEC1AF08DEC10F04F0ECD
:10327000E8CF91F186EF1AF0409B93EC10F040A15B
:1032800047EF19F0500EE8CF91F16DEF12F040AD1D
:103290004DEF19F0550EE8CF91F186EF1AF052502C
:1032A000000AD8A459EF19F0510EE8CF91F15EEF62
:1032B00019F0550EE8CF91F15EEF19F086EF1AF094
:1032C00099EC1AF0520EE8CF91F186EF1AF040AD6A
:1032D0007CEF19F07BEC0DF0409FA68EF86A180E7B
:1032E000F76E000EF66ECCEC1AF0C1EC1AF08DEC15
:1032F00010F0530EE8CF91F186EF1AF0408B93EC6B
:1033000010F040A189EF19F0540EE8CF91F16DEF64
:1033100012F040AD8FEF19F0550EE8CF91F186EF26
:103320001AF05250000AD8A49CEF19F0550EE8CFBD
:1033300091F10F96A1EF19F0550EE8CF91F1A1EFA1
:1033400019F086EF1AF099EC1AF05B0EE8CF91F1C4
:1033500086EF1AF083EC0DF0D8A0B1EF19F099ECDC
:103360001AF040ADCFEF19F07BEC0DF0408FA68E38
:10337000F86A160EF76E260EF66ECCEC1AF0A68ED4
:10338000F86A160EF76E320EF66ECCEC1AF00D0ED1
:1033900067EC0DF09FEC1AF05C0EE8CF91F186EF30
:1033A0001AF083EC0DF0D8A0E7EF19F00D0AD8B4AD
:1033B000D1EF19F0070AD8B4D1EF19F0340AD8A424
:1033C000EAEF19F05D0EE8CF91F1EDEF19F040ADA5
:1033D000EDEF19F0550EE8CF91F186EF1AF083EC7E
:1033E0000DF0D8A00DEF1AF0200AD8A410EF1AF0B3
:1033F000408FA68EF86A160EF76E420EF66ECCEC73
:103400001AF01A0E67EC0DF0DDEC1AF08DEC10F0EE
:103410005E0EE8CF91F113EF1AF040AD13EF1AF002
:10342000550EE8CF91F186EF1AF0409B93EC10F027
:1034300040A120EF1AF05F0EE8CF91F16DEF12F08E
:1034400040AD26EF1AF0550EE8CF91F186EF1AF055
:1034500052500A0AD8A434EF1AF08DEC10F05E0E28
:10346000E8CF91F141EF1AF00A0AD8A43EEF1AF022
:10347000550EE8CF91F10F9641EF1AF0550EE8CFB7
:1034800091F186EF1AF00FB64CEF1AF08986580EBC
:10349000E8CF91F186EF1AF080A457EF1AF0898AED
:1034A0008DEC1AF0560EE8CF91F186EF1AF0899A5A
:1034B0009FEC1AF0590EE8CF91F186EF1AF040AD6B
:1034C00064EF13F0899A93EC1AF0570EE8CF91F15C
:1034D00086EF1AF040AD72EF1AF0550EE8CF91F179
:1034E0007AEF1AF080B47AEF1AF0590E0FA6580E40
:1034F000E8CF91F186EF1AF086EF1AF040AD84EF35
:103500001AF0020EE8CF91F186EF1AF01200C80E01
:10351000946F000E956F409D1200A40E946F010EE3
:10352000956F409D1200280E946F000E956F409D80
:103530001200140E946F000E956F409D1200E80E5D
:10354000946F030E956F409D1200D00E946F070E7E
:10355000956F409D1200F29EF2BEABEF1AF0A00EE6
:10356000946F0F0E956F409DF28E1200F29EF2BE88
:10357000B6EF1AF0980E946F3A0E956F409DF28E4A
:103580001200F29EF2BEC1EF1AF0680E946F420E66
:10359000956F409DF28E12000900F550FF0BD8B4D4
:1035A000D6EF1AF067EC0DF0CCEF1AF040BFDCEF6D
:1035B0001AF00D0E67EC0DF01200A00E946F8C0E39
:1035C000956F409D12002F6F2951D8A4EBEF1AF090
:1035D0004283F8EF1AF0030EEA6E3151E96E2F5173
:1035E000EE6EE9503C0AD8B43C0E3C0A316F290714
:1035F00012003C0E295DD8B403EF1BF0030EEA6EF7
:103600003051E96EEF502F6F12003C0E295DD8A4A7
:103610000DEF1BF042811BEF1BF0030EEA6E3051E1
:10362000E96E30293C0AD8B43C0E3C0A306F292B95
:10363000356BEF502F6F12002F6F030EEA6E305173
:10364000E96E2F51EF6E1200326F3C0E2A5DD8A04A
:103650002DEF1BF042873AEF1BF0030EEA6E345158
:10366000E96E3251EE6EE950780AD8B4440E780A09
:10367000346F2A2B12002A51D8A442EF1BF0428546
:1036800050EF1BF0030EEA6E3351E96EEE50326FCD
:10369000E950780AD8B4440E780A336F2A073251B9
:1036A00012000FA059EF1BF00E0E9E6F9E2F56EFCB
:1036B0001BF01200938851EC1BF0938A51EC1BF025
:1036C0008A98939851EC1BF08A9A939A51EC1BF0CC
:1036D00012008A98939851EC1BF0938A51EC1BF0DE
:1036E000938851EC1BF012009388080E9F6FD890BE
:1036F000A037938A0EB880EF1BF081AA7AEF1BF0F7
:1037000051EC1BF081B8A0818A9A939A51EC1BF07E
:103710009F2F77EF1BF08A980FB293980FA2938890
:10372000938A51EC1BF08A9A939A51EC1BF0938880
:10373000A0511200A06F080E9F6F8A98A0BFA3EF40
:103740001BF0A6EF1BF09388A9EF1BF09398A9EF4D
:103750001BF051EC1BF0938A51EC1BF0A0378A9AB6
:10376000939A51EC1BF09F2F9DEF1BF0938851EC27
:103770001BF0938A51EC1BF00F8482A80F948A9A55
:10378000939A51EC1BF012009488948651EC1BF034
:103790008B98949851EC1BF08B96949651EC1BF0FF
:1037A00012008B9694968B98949851EC1BF094860B
:1037B00051EC1BF0948851EC1BF012009488080E19
:1037C0009F6FD890A03794860EB6EAEF1BF082A6C2
:1037D000E4EF1BF051EC1BF082B8A0818B9694961D
:1037E00051EC1BF09F2FE1EF1BF08B980FB29498D8
:1037F0000FA294880000948651EC1BF000008B9679
:103800000000949651EC1BF08B98949851EC1BF0AF
:10381000A051AA6B1200A06F080E9F6F8B98A0BFDB
:1038200014EF1CF017EF1CF094881AEF1CF094981A
:103830001AEF1CF051EC1BF0948651EC1BF0A037F2
:103840008B96949651EC1BF09F2F0EEF1CF09488F2
:1038500051EC1BF0948651EC1BF00F8482A80F945E
:103860008B9694968B98949851EC1BF012008B8A4F
:1038700063EC0EF0C4EC1BF020340E0BA0090BEC33
:103880001CF01F500BEC1CF01E500BEC1CF0C4EC99
:103890001BF020340E0BA1090BEC1CF012000A0ED9
:1038A000AA6F0F82DEEC1BF012000B0EAA6F0F92B4
:1038B000DEEC1BF00F82D1EC1BF08B9A51EC1BF06D
:1038C00051EC1BF051EC1BF051EC1BF012000EAC54
:1038D00071EF1CF0ACA26AEF1CF08B928B80480E4B
:1038E000AD6EA60EA66F24EC1BF0A151A62724EC0A
:1038F0001BF0A251A62724EC1BF09C0EE16E010EDA
:10390000E26EE550A62724EC1BF0E550A62724EC38
:103910001BF0E550A62724EC1BF0E550E550A62748
:1039200024EC1BF0E550A62724EC1BF0E550A6275D
:1039300024EC1BF011EE11F0E650A62724EC1BF04E
:10394000E650A62724EC1BF0E650A62724EC1BF03B
:10395000E650A62724EC1BF0E650A62724EC1BF02B
:10396000E650A62724EC1BF0E650A62724EC1BF01B
:10397000E650A62724EC1BF0E650A62724EC1BF00B
:10398000A61D010F24EC1BF0200EE3EC1AF00EAC88
:10399000D1EF1CF0ACA2CAEF1CF08B928B80680EAA
:1039A000AD6E1200776F240E7719D8B4766BFB6A70
:1039B000390EFA6E7635E8343C0BC20FD8B0FA2ACD
:1039C000F96E01EF1DF00AEF1DF042EF1DF069EFF7
:1039D0001DF098EF1DF009EF1FF009EF1FF009EF40
:1039E0001FF009EF1FF009EF1FF009EF1FF009EFBB
:1039F0001FF009EF1FF009EF1FF009EF1FF009EFAB
:103A00001FF004EE00F07751EF6E0C90010E766F10
:103A10000EEF1FF004EE01F07751EF6E786F78AF84
:103A200014EF1DF009EF1FF0020E4C6FFB6A3A0E07
:103A3000FA6E7839E834E8340C0B420FD8B0FA2A21
:103A4000F96E2DEF1DF02DEF1DF029EF1DF031EF78
:103A50001DF0000E796F3EEF1DF0010E796F35EF0E
:103A60001DF0030E796F35EF1DF078BD3CEF1DF0B2
:103A700078510F0B010F79273EEF1DF0020E766F84
:103A80000EEF1FF07951D8A44AEF1DF0030E766FA8
:103A9000D7EF1CF00CA052EF1DF00C902F0E775FAB
:103AA0005AEF1DF02F0E775DD8A45AEF1DF00C8051
:103AB00067EF1DF004EE00F04C51E96E7751EE6EA9
:103AC000E9504C6F792F67EF1DF0030E766F0EEF04
:103AD0001FF00CA071EF1DF00C902F0E775F79EFA7
:103AE0001DF02F0E775DD8A479EF1DF00C8096EFB6
:103AF0001DF004EE00F04C51E96E7751EF6E000EB0
:103B0000AB6F000E4C5D796F790704EE01F0EE505B
:103B1000AB27792F87EF1DF0AB1D010FEF5CD8A409
:103B200009EF1FF0040E766FD7EF1CF00EEF1FF0B9
:103B30000C8404EE01F0EF500F0B010F796FFB6A5C
:103B40003B0EFA6EEF38E834E8340C0B540FD8B063
:103B5000FA2AF96EB2EF1DF00CEF1EF07CEF1EF0AA
:103B6000BCEF1EF08A86EF50786F51EC1BF004EE2C
:103B700002F05AEC1BF0D00E9AEC1BF0EE50AC6F3A
:103B80009AEC1BF078BDEBEF1DF0EE50AD6FAC5131
:103B9000000AD8A4D0EF1DF07F0EAD17DAEF1DF0AC
:103BA000070AD8A4D8EF1DF0100EAD6FDAEF1DF0A4
:103BB000DAEF1DF0AC2BAD519AEC1BF0792FC5EF6D
:103BC0001DF069EC1BF08A9651EC1BF014EC1FF011
:103BD0000C8607EF1FF0230EE8CF00F4790590095B
:103BE000E8CF01F404EE02F05AEC1BF0D10E9AEC8F
:103BF0001BF00F8274EC1BF0EE6E792FF9EF1DF0C5
:103C00000F9274EC1BF069EC1BF08A9651EC1BF0E0
:103C10001EEC1FF007EF1FF004EE02F0EFAE13EF03
:103C20001EF049EF1EF011EE00F0EE50E126D8B084
:103C3000E22A01C4E8FFE8BC37EF1EF0020EE15CA7
:103C4000D8A028EF1EF0200EE15CD8A02CEF1EF0CB
:103C5000EE50E6502EEF1EF0EE50E66E792F1EEF7E
:103C60001EF06DEC1FF014EC1FF007EF1FF0230E99
:103C7000E8CF00F479059009E8CF01F404EE02F0F2
:103C8000E650EE6E792F40EF1EF01EEC1FF007EFAE
:103C90001FF0EE50A96E78BD66EF1EF0A69EA69CA2
:103CA000A684EE50A86EF29E550EA76EAA0EA76EC1
:103CB000A682F28EA6B25AEF1EF0A92A792F51EFF2
:103CC0001EF0A69414EC1FF007EF1FF0230EE8CFB0
:103CD00000F479059009E8CF01F404EE02F0A69E05
:103CE000A69CA680A850EE6EA92A792F71EF1EF02F
:103CF0001EEC1FF007EF1FF0FB6A3D0EFA6EEF504F
:103D0000E834E8343C0B0E0FD8B0FA2AF96EA9EF6C
:103D10001EF0A9EF1EF0A7EF1EF0A9EF1EF0A9EF0D
:103D20001EF0AFEF1EF0A9EF1EF0A9EF1EF0ABEFF3
:103D30001EF0ADEF1EF0B3EF1EF0A9EF1EF0A9EFDD
:103D40001EF0B8EF1EF0A9EF1EF0A9EF1EF007EF6E
:103D50001FF007EF1FF007EF1FF007EF1FF014EC45
:103D60001FF007EF1FF00F8614EC1FF007EF1FF096
:103D700014EC1FF007EF1FF0EE50786FEE50206E3E
:103D8000EE501F6EEE501E6E78BDF0EF1EF08B8A67
:103D900051EC1BF0C4EC1BF020340E0BA0090BEC13
:103DA0001CF01F500BEC1CF01E500BEC1CF0EE50E6
:103DB0000BEC1CF0792FD7EF1EF0D1EC1BF063EC6D
:103DC0000EF063EC0EF063EC0EF063EC0EF063ECBF
:103DD0000EF08B9A51EC1BF014EC1FF007EF1FF064
:103DE000230EE8CF00F479059009E8CF01F404EE42
:103DF00002F037EC1CF04FEC1CF0EE6E792FFBEF6D
:103E00001EF055EC1CF01EEC1FF007EF1FF009EF41
:103E10001FF0766B7BEC0DF00EEF1FF083EC0DF0D6
:103E2000D8B0D2EC1CF01200230E67EC0DF08A0E15
:103E300067EC0DF0760E67EC0DF0120004EE01F069
:103E4000796B01C4E8FFE838070BD8B431EF1FF0F5
:103E50004C6F01C4E8FF0F0B010F79274C2F2DEF9A
:103E60001FF0010F796F000EAB6FEE50AB27792F6B
:103E700035EF1FF0AB1D010FEE6EE9504C6F14EEE5
:103E800000F00C820C900CA04BEF1FF00C90E65051
:103E90002F0F65EF1FF00CB263EF1FF0230EE75CEE
:103EA000D8B45DEF1FF0240EE75CD8B45DEF1FF0CF
:103EB0002F0EE75CD8A463EF1FF00C802F0E67EC89
:103EC0000DF043EF1FF00C92E65067EC0DF0E1505F
:103ED0004C5DD8A443EF1FF01200A56B000ED3EC8D
:103EE0000EF05A0AD8B47AEF1FF0FF0AD8B482EF66
:103EF0001FF0FF00400E7B6F000E7C6FA50E7E6FE3
:103F00008AEF1FF0000E7B6F400E7C6F5A0E7E6FA3
:103F10008AEF1FF0020E7B25D3EC0EF0025DD8B4C1
:103F200095EF1FF00251DCEC0EF0030E7B25D3EC75
:103F30000EF0035DD8B4A0EF1FF00351DCEC0EF0DF
:103F4000040E7B25D3EC0EF0045DD8B4ABEF1FF06C
:103F50000451DCEC0EF0050E7B25D3EC0EF0055D74
:103F6000D8B4B6EF1FF00551DCEC0EF0060E7B2541
:103F7000D3EC0EF0065DD8B4C1EF1FF00651DCECB7
:103F80000EF0070E7B25D3EC0EF0075DD8B4CCEF16
:103F90001FF00751DCEC0EF0080E7B25D3EC0EF081
:103FA000085DD8B4D7EF1FF00851DCEC0EF0090E15
:103FB0007B25D3EC0EF0095DD8B4E2EF1FF0095178
:103FC000DCEC0EF00A0E7B25D3EC0EF00A5DD8B4C3
:103FD000EDEF1FF00A51DCEC0EF00B0E7B25D3EC5D
:103FE0000EF00B5DD8B4F8EF1FF00B51DCEC0EF0C7
:103FF0000C0E7B25D3EC0EF00C5DD8B403EF20F053
:104000000C51DCEC0EF00D0E7B25D3EC0EF00D5DAB
:10401000D8B40EEF20F00D51DCEC0EF00E0E7B2527
:10402000D3EC0EF00E5DD8B419EF20F00E51DCEC9D
:104030000EF00F0E7B25D3EC0EF00F5DD8B424EFFD
:1040400020F00F51DCEC0EF0100E7B25D3EC0EF0BF
:10405000105DD8B42FEF20F01051DCEC0EF0110EF3
:104060007B25D3EC0EF0115DD8B43AEF20F011515E
:10407000DCEC0EF0120E7B25D3EC0EF0125DD8B402
:1040800045EF20F01251DCEC0EF0130E7B25D3EC43
:104090000EF0135DD8B450EF20F01351DCEC0EF0AD
:1040A000140E7B25D3EC0EF0145DD8B45BEF20F03A
:1040B0001451DCEC0EF0150E7B25D3EC0EF0155DE3
:1040C000D8B466EF20F01551DCEC0EF0160E7B250F
:1040D000D3EC0EF0165DD8B471EF20F01651DCEC85
:1040E0000EF0170E7B25D3EC0EF0175DD8B47CEFE5
:1040F00020F01751DCEC0EF0180E7B25D3EC0EF0FF
:10410000185DD8B487EF20F01851DCEC0EF0190ED2
:104110007B25D3EC0EF0195DD8B492EF20F0195145
:10412000DCEC0EF01A0E7B25D3EC0EF01A5DD8B441
:104130009DEF20F01A51DCEC0EF01B0E7B25D3EC2A
:104140000EF01B5DD8B4A8EF20F01B51DCEC0EF094
:104150001C0E7B25D3EC0EF01C5DD8B4B3EF20F021
:104160001C51DCEC0EF01D0E7B25D3EC0EF01D5D1A
:10417000D8B4BEEF20F01D51DCEC0EF01E0E7B25F6
:10418000D3EC0EF01E5DD8B4C9EF20F01E51DCEC6C
:104190000EF01F0E7B25D3EC0EF01F5DD8B4D4EFCC
:1041A00020F01F51DCEC0EF0010E7C25D3EC0EF05C
:1041B0007D6F010E7B25D3EC0EF07D2BFF0E7D195C
:1041C000D8B47D2B7D51DCEC0EF0000ED3EC0EF05C
:1041D0007E51DCEC0EF01200000ED3EC0EF05A0A09
:1041E000D8B427EF21F0FF0AD8B42AEF21F0010E4E
:1041F000D3EC0EF0806F010E400FD3EC0EF0816F08
:10420000FF0E8019D8B42AEF21F0FF0E8119D8B41F
:1042100027EF21F0FE0E8019D8B421EF21F0FE0E19
:104220008119D8B41BEF21F08051815DD8A027EF10
:1042300021F02AEF21F08051D8A42AEF21F027EFB6
:1042400021F08151D8A427EF21F02AEF21F0000EB0
:104250002DEF21F0400E2DEF21F07F6F020E7F2514
:10426000D3EC0EF0026F030E7F25D3EC0EF0036F3C
:10427000040E7F25D3EC0EF0046F050E7F25D3ECE2
:104280000EF0056F060E7F25D3EC0EF0066F070EBD
:104290007F25D3EC0EF0076F080E7F25D3EC0EF0D0
:1042A000086F090E7F25D3EC0EF0096F0A0E7F25EB
:1042B000D3EC0EF00A6F0B0E7F25D3EC0EF00B6FD4
:1042C0000C0E7F25D3EC0EF00C6F0D0E7F25D3EC7A
:1042D0000EF00D6F0E0E7F25D3EC0EF00E6F0F0E4D
:1042E0007F25D3EC0EF00F6F100E7F25D3EC0EF070
:1042F000106F110E7F25D3EC0EF0116F120E7F257B
:10430000D3EC0EF0126F130E7F25D3EC0EF0136F6B
:10431000140E7F25D3EC0EF0146F150E7F25D3EC11
:104320000EF0156F160E7F25D3EC0EF0166F170EDC
:104330007F25D3EC0EF0176F180E7F25D3EC0EF00F
:10434000186F190E7F25D3EC0EF0196F1A0E7F250A
:10435000D3EC0EF01A6F1B0E7F25D3EC0EF01B6F03
:104360001C0E7F25D3EC0EF01C6F1D0E7F25D3ECA9
:104370000EF01D6F1E0E7F25D3EC0EF01E6F1F0E6C
:104380007F25D3EC0EF01F6F1200FFFFFFFFFFFF32
:10439000FFFFFFFFFFFFFFFFFFFFFFFFFFFFFFFF2D
:1043A000FFFFFFFFFFFFFFFFFFFFFFFFFFFFFFFF1D
:1043B000FFFFFFFFFFFFFFFFFFFFFFFFFFFFFFFF0D
:1043C000FFFFFFFFFFFFFFFFFFFFFFFFFFFFFFFFFD
:0200000400F00A
:100000005A634C37303700000000AA00000400009B
:1000100004000000FF00FFFF00000000000000FFE0
:10002000FF00FFFFFFFFFFFFFFFFFFFFFFFFFFFFDF
:10003000FFFFFFFFFFFFFFFFFFFFFFFFFFFFFFFFD0
:100040005A62FFFFFFFFFFFFFFFFFFFFFFFFFFFF02
:10005000FFFFFFFFFFFFFFFFFFFFFFFFFFFFFFFFB0
:10006000FFFFFFFFFFFFFFFFFFFFFFFFFFFFFFFFA0
:10007000FFFFFFFFFFFFFFFFFFFFFFFFFFFFFFFF90
:100080004338473253435241544348504144FFFFA1
:10009000FFFFFFFFFFFFFFFFFFFFFFFFFFFFFFFF70
:1000A000FFFFFFFFFFFFFFFFFFFFFFFFFFFFFFFF60
:1000B000FFFFFFFFFFFFFFFFFFFFFFFFFFFFFFFF50
:1000C000FFFFFFFFFFFFFFFFFFFFFFFFFFFFFFFF40
:1000D000FFFFFFFFFFFFFFFFFFFFFFFFFFFFFFFF30
:1000E000FFFFFFFFFFFFFFFFFFFFFFFFFFFFFFFF20
:1000F000FFFFFFFFFFFFFFFFFFFFFFFFFFFFFFFF10
:020000040030CA
:0E0000000023003C009D80000C800FE00F40AC
:020000040020DA
:08000000FFFFFFFFFFFFFFFF00
:00000001FF
